:020000040000FA
:100000001629FF3FFF3FFF3FF000030EF1000408F9
:10001000F2000A08F30083018A01A30A8B18112851
:10002000102883018B10060EF400F40CF50DF40C6F
:10003000F50DF40CF50DF40CF50D75080F39A8004D
:1000400073088A0072088400710E8300F00E700E2F
:100050000900FF3FFF3FFF3FFF3FFF3FFF3FFF3FE5
:10006000FF3FFF3FFF3FFF3FFF3FFF3FFF3FFF3FA0
:10007000FF3FFF3FFF3FFF3FFF3FFF3FFF3FFF3F90
:10008000FF3FFF3FFF3FFF3FFF3FFF3FFF3FFF3F80
:10009000FF3FFF3FFF3FFF3FFF3FFF3FFF3FFF3F70
:1000A000FF3FFF3FFF3FFF3FFF3FFF3FFF3FFF3F60
:1000B000FF3FFF3FFF3FFF3FFF3FFF3FFF3FFF3F50
:1000C000FF3FFF3FFF3FFF3FFF3FFF3FFF3FFF3F40
:1000D000FF3FFF3FFF3FFF3FFF3FFF3FFF3FFF3F30
:1000E000FF3FFF3FFF3FFF3FFF3FFF3FFF3FFF3F20
:1000F000FF3FFF3FFF3FFF3FFF3FFF3FFF3FFF3F10
:10010000FF3FFF3FFF3FFF3FFF3FFF3FFF3FFF3FFF
:10011000FF3FFF3FFF3FFF3FFF3FFF3FFF3FFF3FEF
:10012000FF3FFF3FFF3FFF3FFF3FFF3FFF3FFF3FDF
:10013000FF3FFF3FFF3FFF3FFF3FFF3FFF3FFF3FCF
:10014000FF3FFF3FFF3FFF3FFF3FFF3FFF3FFF3FBF
:10015000FF3FFF3FFF3FFF3FFF3FFF3FFF3FFF3FAF
:10016000FF3FFF3FFF3FFF3FFF3FFF3FFF3FFF3F9F
:10017000FF3FFF3FFF3FFF3FFF3FFF3FFF3FFF3F8F
:10018000FF3FFF3FFF3FFF3FFF3FFF3FFF3FFF3F7F
:10019000FF3FFF3FFF3FFF3FFF3FFF3FFF3FFF3F6F
:1001A000FF3FFF3FFF3FFF3FFF3FFF3FFF3FFF3F5F
:1001B000FF3FFF3FFF3FFF3FFF3FFF3FFF3FFF3F4F
:1001C000FF3FFF3FFF3FFF3FFF3FFF3FFF3FFF3F3F
:1001D000FF3FFF3FFF3FFF3FFF3FFF3FFF3FFF3F2F
:1001E000FF3FFF3FFF3FFF3FFF3FFF3FFF3FFF3F1F
:1001F000FF3FFF3FFF3FFF3FFF3FFF3FFF3FFF3F0F
:10020000F40001308A0074080F3982074434313415
:100210003234333434343534363437343834393492
:1002200030342A34233441344234433483018A0144
:100230008B016400103085000030860007309F007D
:1002400083164F308100E0308500FF308600831236
:1002500083018E018F0130309000830183167C3042
:100260009200831226309200830183161930990080
:10027000243098008312803098008301A401E001AB
:10028000A501A601A701A801A9016430A20083016C
:100290008B018C0183168C01830190308B008301CC
:1002A0008A018C1C4F298C1064008301E00803191B
:1002B0005F2960306007840000089900E0030310A4
:1002C00006180314A50DA60D241F7D29A41B6D2956
:1002D00025080339031D8C2974292508031D8C2941
:1002E00026080F39031D8C29241329080F39A41A55
:1002F0008038E1000130E0008C2925080339033CF7
:10030000031D8C29241728080F39A9001038A41AB6
:100310008038E1000130E0008301061C91290512BC
:1003200092290516A20BA0296430A200861D9A29E5
:10033000A4179B29A413861C9F29A416A029A412E4
:100340004F29FF3FFF3FFF3FFF3FFF3FFF3FFF3F83
:10035000FF3FFF3FFF3FFF3FFF3FFF3FFF3FFF3FAD
:10036000FF3FFF3FFF3FFF3FFF3FFF3FFF3FFF3F9D
:10037000FF3FFF3FFF3FFF3FFF3FFF3FFF3FFF3F8D
:10038000FF3FFF3FFF3FFF3FFF3FFF3FFF3FFF3F7D
:02400E00653F0C
:084000000800010001000100AD
:00000001FF
